:040000000C946901F2
:04004C000C941802F6
:040058000C9472038F
:1400700000002000002A0000532079206C20762061206920FA
:140084006E20202042206920732073206F206E206E20652059
:140098007420742065000056203A2031202E203000004420C4
:1400AC0044204420202045204520452045202042204220427E
:1400C000202020205520552055202020204720472047202098
:1400D40020204720472047202020452045204520452020525D
:1400E800202020202052000044202020204420204520202025
:1400FC002020202020422020202042202055202020202055C2
:140110002020472020202020472020472020202020472020BF
:140124004520202020202020205220202020522000004420DA
:1401380020202044202045204520452020202042202020425C
:14014C00202020552020202020552020472020472047202040
:140160002047202047204720202045204520452020202052F5
:14017400205220522020000044202020204420204520202066
:14018800202020202042202020204220205520202020205535
:14019C00202047202020202020202047202020202020202081
:1401B00045202020202020202052202020205220000044204E
:1401C400442044202020452045204520452020422042204265
:1401D8002020205520202020205520202047204720472020B4
:1401EC00202047204720472020204520452045204520205244
:14020000205220522020000041202020202020204120202004
:140214002056202020202020205220202020205220202020BC
:140228002020202020200000204120412041204120202020FE
:14023C0056205620202020202052202020205220202020205E
:140250002020202020200000202041202020412020202056E2
:1402640020202056202020202052205220522020202020203A
:140278002020202020200000202020412041202020205620BA
:14028C00202020205620202020522020202052202020202044
:1402A0002020202020200000202020204120202020562020B3
:1402B4002020202020562020205220522052202020202020EA
:0902C8002020202020200000016C
:1402D200CFEFD4E0CDBFDEBFCE51D0400AEA08830024E1E0EA
:1402E600F1E013E0E835F10711F00192FBCF0083E0EDF2E0AB
:1402FA00A0E0B1E012E000E00BBFE13DF10721F0C8953196F8
:14030E000D92F9CF0E948C01FFCF22977894CAD088EA92E034
:140322009983888323E008E1D7D080E892E09983888324E008
:1403360008E1D0D088E592E09983888325E008E1C9D080E33A
:14034A0092E09983888326E008E1C2D088E092E09983888384
:14035E0027E008E1BBD082EC91E0998388832AE006E0B4D096
:140372008CE791E0998388832BE006E0ADD086E391E0998308
:1403860088832CE006E0A6D080EF90E0998388832DE006E0F7
:14039A009FD08AEA90E0998388832EE006E098D08FE990E091
:1403AE009983888324E103E291D088E790E09983888325E1BD
:1403C20007E18AD0442714C085E790E09983888321E1042F6E
:1403D6000A5F80D018D082E790E09983888321E1042F0A5FD4
:1403EA00015076D00ED04395443450F382E790E099838883F7
:1403FE00222700276BD00DD0FFCF229608950027112702C01F
:140412000F5F1F4F0033E5E71E07D0F3089588E98AB986EA52
:1404260080BD222420BC29B808950A921A922A923A924A9239
:14043A005A926A927A928A929A920A931A932A933A934A93C1
:14044E008A939A93AA93BA93EA93FA930FB60A924A935C9989
:1404620004C05B9902C05A9B05C04CB189B18F5F89B905C026
:140476004CB14F3710F4042FF7D0499109900FBEF991E991AD
:14048A00B991A99199918991499139912991199109919990CB
:14049E008990799069905990499039902990199009901895FC
:1404B2002C9706D122242CBE89E180B922B888E281B986E8DD
:1404C6008CBF80E790E0998388832227002702D02C96089538
:1404DA00AA92CA92C22EA02E2A97AA20F9F4CC20E9F48BE10B
:1404EE0088838BE5898382E38A838AE48B8322242C828E0102
:14050200A6D08BE188838BE5898381E38A838BE38B8381E32B
:140516008C8388E48D8322242E828E0196D02BC08BE18883F9
:14052A008BE589831AE00C2D0E94AD03802F805D8A831AE029
:14053E000C2D0E94AB03802F805D8B838BE38C831AE00A2DD8
:140552000E94AD03802F805D8D831AE00A2D0E94AB03802F77
:14056600805D8E8386E68F83222428868E016DD00C851D8522
:14057A0059D02A96C990A9900895AA92CA92C22EA02E2A973E
:14058E00AA20F9F4CC20E9F48BE188838BE5898382E38A8374
:1405A2008AE48B8322242C828E0151D08BE188838BE5898332
:1405B60081E38A838BE38B8381E38C8388E48D8322242E825F
:1405CA008E0141D02BC08BE188838BE589831AE00C2D0E94CA
:1405DE00AD03802F805D8A831AE00C2D0E94AB03802F805DB1
:1405F2008B838BE38C831AE00A2D0E94AD03802F805D8D834B
:140606001AE00A2D0E94AB03802F805D8E8386E68F832224FE
:14061A0028868E0118D00C851D8515D02A96C990A9900895A0
:14062E004A935A93A80106C01A014F5F5F4FF101049116D09B
:14064200FA0124902220B1F7599149910895AA92BA925801C9
:1406560004C0F50101915F0107D0F50120802220C1F7B99034
:14066A00A990089501C0A8958EE490E020900203309003034B
:14067E0082159305B0F3E0910603F09107030193F093070370
:14069200E093060388E593E0E817F90731F488E093E09093D6
:1406A60007038093060380910203909103030196909303031D
:1406BA00809302030D9A089588E093E09093070380930603AC
:1406CE009093050380930403222433243092030320920203B7
:1406E20008952A923A928A939A93EA93FA932FB62A9220903A
:1406F600020330900303222011F43320F9F0E0910403F091A9
:14070A0005032190F0930503E093040323B888E593E0E81763
:14071E00F90731F488E093E09093050380930403809102036C
:14073200909103030197909303038093020301C00D98299094
:140746002FBEF991E99199918991399029901895689401C07E
:14075A00E8942A93FA92EA92FF24EE2420E1000FFF1CEE1CE0
:14076E00E11610F0E11A03952A95B9F70EF40E2DE990F9903F
:04078200299108951C
:00000001FF
